:020000040000FA
:06000000D43001303A2863
:08000800A000030EA100831209
:1000100005191128831601178312B2308100B1012E
:100020002C2883160113831203140B190310A80D37
:10003000A90DAA0DAB0DAC0DAC16FF302C02031DA3
:100040002C28FA302B02031D2C2832152A08AF0069
:100050002908AE002808AD008B100B11210E83007B
:06006000A00E200E0900B5
:04006600003400342E
:0C007400203084008001840A80300402E7
:10008000031C3C28D52183160C308505870183127B
:10009000850187010730990000309A0010308316DF
:1000A0008E008312603083168F0083120030831617
:1000B000910000008312C830831681008312313012
:1000C0009000003083168C00831210308B00C12208
:1000D00081018E018F010B118B100B108C018B177E
:1000E0007F2032198B20B40B7D280310851903144F
:1000F000BA0DF0303A02031934212023702864002D
:100100003310B10A311F8A28AC01AB01AA01A90141
:10011000A801B101080032110130B7008B13203063
:10012000370783169B001C141A088312A400103092
:10013000370783169B001C141A088312A300A6001D
:100140000230A6060030370783169B001C141A08DD
:100150008312A200A7000130A7068B17331CB62814
:1001600022090339A200A309A409A50924082F0222
:10017000031D2E2923082E02031D2E2922082D02DD
:10018000031D2E2901303702031DCB283E18CB2832
:100190003E143F14F72102303702031DD428BE1845
:1001A000D428BE143F14032203303702031DDD2878
:1001B0003E19DD283E153F140F2204303702031D7F
:1001C000E628BE19E628BE153F141B22053037026B
:1001D000031DEF283E1AEF283E163F142722063053
:1001E0003702031DF828BE1AF828BE163F14332222
:1001F00007303702031D01293E1B01293E173F141A
:100200003F2208303702031D0A29BE1B0A29BE17E8
:100210003F144A2209303702031D13295D181329A0
:100220005D143F1455220A303702031D1C29DD18C6
:100230001C29DD143F1460220B303702031D2529D1
:100240005D1925295D153F146B220C303702031D03
:100250002E29DD192E29DD153F147622B70A0D301F
:100260003702031808008E280130B600B400B5002C
:10027000B70085018701B213BE227F20B40B4D2940
:10028000031085190314BA0DF0303A0203197529C9
:10029000B50B4D299630B5008121321D3D29321113
:1002A000331C57292D090339AD00AE09AF092F1CA6
:1002B0003D292D08300203193D292D08B0002E1EBE
:1002C0003D298B1320303707BC002F08BB00C0210D
:1002D00010303707BC002E08BB00C02100303707A4
:1002E000BC002D08BB00C0218B1785018701B70A10
:1002F000B6010130B5000D303702031C3D29C12283
:100300000800013037020319822202303702031934
:1003100087220330370203198C2204303702031975
:10032000912205303702031996220630370203194D
:100330009B22073037020319A02208303702031925
:10034000A522093037020319AA220A3037020319FD
:10035000AF220B3037020319B4220C3037020319D5
:10036000B92208003F1C08003F101030BC003E08B6
:10037000BB00C0213030BC005D08BB00C0210800BC
:100380008B133B0883161C159A0083123C088316B6
:100390009B0055309D00AA309D009C1464009C1861
:1003A000CE291C1183128B170800831600309B0086
:1003B0001C141A088312BD00831610309B001C14F5
:1003C0001A088312BE00831630309B001C141A08D2
:1003D0008312DD00FF30C800CA15CB15CC15CD1532
:1003E000CE15CF15D015D115D215D3150800C130B3
:1003F000BE05FF30DD055F140C30C405C0000030C1
:10040000C2005E100800C230BE05FF30DD055F147B
:100410000330C405C0000030C2005E100800C430C4
:10042000BE05FF30DD055F141330C405C000003089
:10043000C2005E100800C830BE05FF30DD055F1445
:100440000930C405C0000030C2005E100800D03082
:10045000BE05FF30DD055F141930C405C000003053
:10046000C2005E100800E030BE05FF30DD055F14FD
:100470000030C405C0000030C2005E1008007F30AC
:10048000BE050030DD05DF146030C505C100003059
:10049000C3000800BF30BE050030DD05DF14183092
:1004A000C505C1000030C30008003F30BE05013063
:1004B000DD05DF149830C505C1000030C300080019
:1004C0003F30BE050230DD05DF144830C505C100F0
:1004D0000030C30008003F30BE050430DD05DF14E6
:1004E000C830C505C1000030C30008003F30BE055C
:1004F0000830DD05DF140030C505C1000030C30041
:1005000008000800033085060030870608003030F8
:1005100085060030870608003030850602308706E1
:100520000800123085060030870608001230850664
:10053000023087060800333085060230870608003F
:10054000003085063030870608000030850605300B
:1005500087060800003085060D3087060800003049
:100560008506143087060800003085061C30870693
:100570000800003085063D30870608003E188222BC
:1005800008003E18F721BE1803223E190F22BE199B
:100590001B223E1A2722BE1A33223E1B3F22BE1BBD
:1005A0004A225D185522DD1860225D196B22DD1983
:1005B00076220800B601B401B5013D1CE22ABD0156
:1005C000BD14E42ABD013D143D08B6006400E82ACC
:1005D000E92AEA2AEB2AEC2AFF30B51B8500B51F71
:1005E0008501B40BE62AB50BE62A0310B60CB60853
:1005F000031DE62A0030BC003D08BB00C0210800F6
:1006000005125C180516DC1C8512DC1885165C1DAD
:1006100005105C190514DC1D8510DC1985145C1EA1
:1006200087105C1A8714DC1E0711DC1A07155C1F83
:1006300007105C1B0714DC1F8712DC1B87160800E1
:100640008F08031908008F0178308E00C80F682DBD
:10065000C80A420843040319332B4208C600C201EA
:100660004308C700C301DE195C2B441C5C2B461CED
:100670004D2BCA1C3E2BCA014A156A2B4A1D432B1F
:10068000CA01CA156A2BCA1D482BCA014A166A2B11
:100690004A1E6A2BCA01CA146A2B4A1D522BCA0170
:1006A0004A166A2BCA1D572BCA014A166A2B4A1EC4
:1006B0006A2BCA01CA146A2BCA1C612BCA014A15CB
:1006C0006A2B4A1D662BCA01CA156A2B4A1E6A2B61
:1006D000CA014A15DE19932BC41C932BC61C842B0C
:1006E000CB1C752BCB014B15A12B4B1D7A2BCB01B2
:1006F000CB15A12BCB1D7F2BCB014B16A12B4B1E5A
:10070000A12BCB01CB14A12B4B1D892BCB014B165D
:10071000A12BCB1D8E2BCB014B16A12B4B1EA12B3E
:10072000CB01CB14A12BCB1C982BCB014B15A12BB0
:100730004B1D9D2BCB01CB15A12B4B1EA12BCB0110
:100740004B15DE19CA2B441DCA2B461DBB2BCC1CD6
:10075000AC2BCC014C15D82B4C1DB12BCC01CC159E
:10076000D82BCC1DB62BCC014C16D82B4C1ED82B1D
:10077000CC01CC14D82B4C1DC02BCC014C16D82B43
:10078000CC1DC52BCC014C16D82B4C1ED82BCC0124
:10079000CC14D82BCC1CCF2BCC014C15D82B4C1DFA
:1007A000D42BCC01CC15D82B4C1ED82BCC014C15FE
:1007B000DE19022CC41D022CC61DF32BCD1CE42B0C
:1007C000CD014D155E13102C4D1DE92BCD01CD151E
:1007D000102CCD1DEE2BCD014D16102C4D1E102CC6
:1007E000CD01CD14102C4D1DF82BCD014D16102C24
:1007F000CD1DFD2BCD014D16102C4D1E102CCD0105
:10080000CD14102CCD1C072CCD014D15102C4D1DD9
:100810000C2CCD01CD15102C4D1E102CCD014D15DD
:10082000DE193B2C5E1B3B2C441E3B2C461E2C2C05
:10083000CE1C1D2CCE014E15492C4E1D222CCE0156
:10084000CE15492CCE1D272CCE014E16492C4E1EFE
:10085000492CCE01CE14492C4E1D312CCE014E1602
:10086000492CCE1D362CCE014E16492C4E1E492C3D
:10087000CE01CE14492CCE1C402CCE014E15492C55
:100880004E1D452CCE01CE15492C4E1E492CCE01B5
:100890004E15DE19722CC51D722CC71D632CCF1C82
:1008A000542CCF014F15802C4F1D592CCF01CF1543
:1008B000802CCF1D5E2CCF014F16802C4F1E802C1C
:1008C000CF01CF14802C4F1D682CCF014F16802CE8
:1008D000CF1D6D2CCF014F16802C4F1E802CCF01C9
:1008E000CF14802CCF1C772CCF014F15802C4F1D9F
:1008F0007C2CCF01CF15802C4F1E802CCF014F15A3
:10090000DE19A92C451EA92C471E9A2CD01C8B2C15
:10091000D0015015B72C501D902CD001D015B72CFC
:10092000D01D952CD0015016B72C501EB72CD001DD
:10093000D014B72C501D9F2CD0015016B72CD01DB1
:10094000A42CD0015016B72C501EB72CD001D014B7
:10095000B72CD01CAE2CD0015015B72C501DB32C89
:10096000D001D015B72C501EB72CD0015015DE1970
:10097000E02CC51EE02CC71ED12CD11CC22CD101ED
:100980005115EE2C511DC72CD101D115EE2CD11DC6
:10099000CC2CD1015116EE2C511EEE2CD101D114CC
:1009A000EE2C511DD62CD1015116EE2CD11DDB2C75
:1009B000D1015116EE2C511EEE2CD101D114EE2C8A
:1009C000D11CE52CD1015115EE2C511DEA2CD10181
:1009D000D115EE2C511EEE2CD1015115DE19182D1A
:1009E000451F182D471F092DD21CFA2CD201521574
:1009F000DE13262D521DFF2CD201D215262DD21D1D
:100A0000042DD2015216262D521E262DD201D214AB
:100A1000262D521D0E2DD2015216262DD21D132D1C
:100A2000D2015216262D521E262DD201D214262D69
:100A3000D21C1D2DD2015215262D521D222DD20160
:100A4000D215262D521E262DD2015215DE19512DFA
:100A5000DE1B512DC51F512DC71F422DD31C332D19
:100A6000D30153155F2D531D382DD301D3155F2DA1
:100A7000D31D3D2DD30153165F2D531E5F2DD30182
:100A8000D3145F2D531D472DD30153165F2DD31D56
:100A90004C2DD30153165F2D531E5F2DD301D3145C
:100AA0005F2DD31C562DD30153155F2D531D5B2D88
:100AB000D301D3155F2D531E5F2DD3015315B221E2
:100AC0004008C4004108C5005E18DE145E1CDE103C
:100AD0004808C9000C304A05031D05120C304B05AF
:100AE000031D85120C304C05031D05100C304D05FF
:100AF000031D85100C304E05031D87100C304F056B
:100B0000031D07110C305005031D07100C30510553
:100B1000031D87120C305205031D07120C305305BC
:100B2000031D871149080E020318C22D12304A0511
:100B3000031D051612304B05031D851612304C059A
:100B4000031D051412304D05031D851412304E058A
:100B5000031D871412304F05031D07151230500571
:100B6000031D071412305105031D8716123052055C
:100B7000031D071612305305031D8715FF30480269
:100B8000031908008F08031D08007F2049080E0282
:100B9000031CC22D18304A05031D051206304A05F4
:100BA000031D051618304B05031D851206304B0535
:100BB000031D851618304C05031D051006304C0525
:100BC000031D051418304D05031D851006304D0515
:100BD000031D851418304E05031D871006304E0581
:100BE000031D871418304F05031D071106304F05EC
:100BF000031D071518305005031D0710063050055A
:100C0000031D071418305105031D871206305105C6
:100C1000031D871618305205031D071206305205B2
:100C2000031D071618305305031D871106305305A1
:060C3000031D87150800FA
:084000000900030007000100A4
:02400E00CC33B1
:10420000010078007A007C007E007B0079007F004E
:104210007D007A0078007E007C007D007F007900C0
:104220004100F200F600FA00FE00F200F600FA008B
:10423000FE00F200F600FA00FE00F200F600FA00BE
:10424000FF00050005000500050009000900090040
:1042500009000D000D000D000D00110011001100EE
:104260000000FF00FF00FF00FF00FF00FF00FF0055
:10427000FF00FF00FF00FF00FF00FF00FF00FF0046
:10428000FF007B00FF00FF00FF00FF00FF00FF00BA
:10429000FF00FF00FF00FF00FF00FF00FF00FF0026
:1042A000FF00FE00FF00FF00FF00FF00FF00FF0017
:1042B000FF00FF00FF00FF00FF00FF00FF00FF0006
:1042C000FF001100FF00FF00FF00FF00FF00FF00E4
:1042D000FF00FF00FF00FF00FF00FF00FF00FF00E6
:1042E000FF00FF00FF00FF00FF00FF00FF00FF00D6
:1042F000FF00FF00FF00FF00FF00FF00FF00DD00E8
:00000001FF
